:020000040800F2
:100000000004022001020008150E0008190E000865
:10001000690E0008190E0008410E000802020008CF
:10002000020200080202000802020008CD250008B2
:100030000202000802020008020200080202000890
:100040000202000802020008020200080202000880
:10005000020200080202000829380008553800088A
:1000600081380008AD380008D938000802020008BD
:100070000202000802020008020200080202000850
:100080000202000802020008020200080202000840
:1000900002020008020200080202000805390008F6
:1000A0000202000802020008020200080202000820
:1000B0004D36000802020008020200080202000891
:1000C0000202000802020008020200080202000800
:1000D0000202000802020008B90F0008020200082C
:1000E0006D3900080202000802020008020200083E
:1000F00002020008020200080202000802020008D0
:1001000002020008020200080202000802020008BF
:1001100002020008020200080202000802020008AF
:10012000020200080202000802020008020200089F
:10013000020200080202000802020008020200088F
:10014000020200080202000802020008312D000825
:10015000020200080202000802020008020200086F
:10016000020200080202000802020008020200085F
:10017000020200080202000802020008020200084F
:100180000202000802020008CD0F00080202000867
:10019000020200080202000802020008020200082F
:1001A000020200080202000802020008020200081F
:1001B000020200080202000802020008020200080F
:1001C00002020008020200080202000802020008FF
:1001D00002020008020200080202000802020008EF
:1001E00002020008020200080202000802020008DF
:1001F00002020008020200080202000802020008CF
:1002000002E000F000F8FEE772B6394880F3088893
:10021000384880F3098838484EF60851CEF200017C
:10022000086040F20000CCF200004EF63471CEF2CD
:1002300000010860BFF34F8FBFF36F8F40F20000E3
:10024000C0F2F0004EF68851CEF200010860BFF314
:100250004F8FBFF36F8F4FF00000E1EE100A4EF6A4
:100260003C71CEF200010860062080F31488BFF3D1
:100270006F8F02F0E9F903F073F94FF055301F4921
:100280001B4A91423CBF41F8040BFAE71C49194A4A
:1002900091423CBF41F8040BFAE71A491A4A1B4B3A
:1002A0009A423EBF51F8040B42F8040BF8E70020D5
:1002B0001749184A91423CBF41F8040BFAE702F093
:1002C00007FA03F0B7F9144C144DAC4203DA54F8B2
:1002D000041B8847F9E700F03FF8114C114DAC4280
:1002E00003DA54F8041B8847F9E702F0EFB900007D
:1002F0000004022000240220000000080000022068
:1003000000040220003E00080024022050240220A5
:1003100050240220183D02200002000800020008BC
:1003200000020008000200082DE9F04F2DED108AB0
:10033000C1F80CD0D0F80CD0BDEC108ABDE8F08F1D
:10034000002383F311882846A047002001F004FE13
:1003500001F0B4FD00DFFEE770B51D4C322300252F
:1003600023706FF07F061F236570A570E5702571FF
:100370006571A571E57125726672A372E57200F070
:1003800067FC20B10F2325726672A372E57202F03A
:10039000FDF8104B984217D00133984241F288344F
:1003A00012BF002500240125002002F0F5F80DB150
:1003B00000F054F800F0CCFC00F096FB204600F072
:1003C000E1F800F04BF8F9E700242546ECE700BF20
:1003D00050240220010007B008B500F003FBA0F193
:1003E00020035842584108BD07B5054B02211B8820
:1003F000ADF8043001A800F061FB03B05DF804FB28
:100400006C3A000810B51148C3680BB101F02AFE20
:100410000F4C104A0D4800234FF47A7101F0E6FDAD
:10042000236813B12368013B2360636813B16368D9
:10043000013B6360084B1B7833B9636823B9022022
:1004400000F038FC3223636010BD00BF5C24022042
:100450007429022005040008702402202DE9F041CF
:10046000414C236801337CD0404D414B2A689A426D
:1004700077D9404B9B6803F1006303F500439A4230
:100480006FD2002000F04AFB3B4B0220187000F0B6
:1004900005FC3A4B1A6C00221A64196E1A66196E22
:1004A000596C5A64596E5A66596E596941F0800107
:1004B0005961596921F0800159615969196941F0FF
:1004C00000511961196921F0005119611B6972B657
:1004D0002B4B1C6024682D68BFF34F8FBFF36F8FC9
:1004E000083BC3F88420BFF34F8F5A6922F480324F
:1004F0005A61BFF34F8FD3F88020C2F3C906C2F30D
:100500004E325201B70743F6E07E02EA0E08384643
:100510003146013948EA000CB1F1FF3FC3F874C21B
:1005200000F14040F5D1203A12F1200FEDD1BFF398
:100530004F8FBFF36F8FBFF34F8FBFF36F8F5A692A
:1005400022F400325A610022C3F85022BFF34F8FC9
:10055000BFF36F8F202383F31188A54684F30888A7
:100560002847BDE8F08100BF008000080480000833
:10057000FF7F00085024022070240220003802402F
:1005800008ED00E02DE9F04FB34B8246B3489C687C
:100590000022C2608FB0202282F31188C2680093CB
:1005A0000AB101F05FFD0023AD4AAC484FF47A7107
:1005B00001F01CFD002383F31188DFF8C0B2BAF10B
:1005C000000F01D0CBF800A0A64FCBF804300025D7
:1005D0003B702E464FF0FF38012000F05FFBBAF170
:1005E000000F00F0C181DBF80030002B40F0BC812F
:1005F0000FB0BDE8F08F0220FFF7EEFE002840F0BC
:10060000AF81994B1B88ADF82430022109A800F076
:1006100055FAE1E74FF47A7000F0E4F9031E019314
:10062000EFDB0220FFF7D8FE81460028E9D0019BCE
:10063000581E0428E5D8DFE800F00310131619004F
:100640000EA8052340F8143D042100F037FA4D466A
:1006500000F074FBFFF7C8FE7FE104217E48F4E759
:1006600004218248F1E704218148EEE71C25284651
:1006700000F056FA04350990042109A800F01EFA8A
:100680002C2DF4D1E3E7002EBBD0002DB9D00220F1
:10069000FFF7A2FE064610B901252E46B1E701205C
:1006A00000F03CFA0220387000F0F8FA00255FFAFA
:1006B00085F9484600F04AFA0135044618B1484623
:1006C00000F054FAF3E7012302203B7000F0D8FA5F
:1006D000009B9B689C4207D2204600F021FA013023
:1006E00040F040810434F3E700243C70CBF8044030
:1006F0003546ADE7002E84D0002D82D00220387020
:1007000000F0CCFA322000F06DF9051EC4DB15F0C4
:100710000306C1D1009A926863199342BCD8B5F51B
:10072000807FB9D8DFF84C91AE420CDA4FF47A7082
:1007300000F058F90390039B002BADDB039B06F8F8
:1007400009300136F0E7C820FFF746FE06460028CC
:10075000A2D02CB9474B4FF0FF32D3F800801A607B
:10076000444B25F003052544A3EB0409AC42BFD05C
:1007700059F80410204600F0D9F9204600F0D0F9CD
:1007800059F80430984240F0ED800434EEE702203E
:10079000FFF722FE00283FF434AF4FF0000AD146A5
:1007A000009B9B689A4537D2BAF1000F17D1B8F178
:1007B000FF3F14D0CDF824802F494B68A3B100220D
:1007C00009A8135C83EA0903DBB2013251F8233034
:1007D000042A83EA1929F4D10AF1040AE0E7504611
:1007E00000F09EF90990E7E71A46082012F0010F81
:1007F0004FEA52021FBF82F06D4282F4380282F447
:10080000034282F020020138F0D141F82320013365
:10081000B3F5807FE8D1D2E70EA8042140F8289DE7
:1008200000F04CF914E70EA8002340F8143D6421B1
:1008300000F010F900287FF4E4AE0220FFF7CCFDB1
:1008400000283FF4DEAE099800F0A2F90EAB43F8A1
:10085000240D04211846E3E7502402205C240220E2
:1008600005040008702402206E3A00085424022077
:1008700058240220742402207425022074290220A6
:100880000EA8002340F8143D642100F0E3F800288E
:100890007FF4B7AE0220FFF79FFD00283FF4B1AE12
:1008A000099800F083F90EAB43F8200DD1E7022040
:1008B000FFF792FD00283FF4A4AE00F07DF90EABE7
:1008C00043F81C0DC5E70220FFF786FD00283FF422
:1008D00098AE09A9142000F075F981460EA80421EC
:1008E00040F8189D00F0EAF8494609A898E74FF447
:1008F0007A70FFF771FD00283FF483AEB8F1FF3F37
:1009000005D1FFF771FD354801F02CFB70E641463B
:10091000002000F00BF9002000F002F98045F0D033
:100920002F4B6FE60EA8002340F8143D642100F021
:1009300091F800287FF465AE0220FFF74DFD0028F6
:100940003FF45FAEFFF750FD41F2883001F00AFB43
:10095000099800F03FFA00F0F1F94FF0000A3BE689
:10096000064675E63546DBE7002000F03BF80390CD
:10097000039B002BFFF633AE012000F081F9039BAF
:10098000213B122B3FF628AE01A252F823F000BF04
:10099000F70500081506000887060008D9050008B5
:1009A000D9050008D9050008F5060008D905000892
:1009B0008F0700082708000881080008AF08000812
:1009C000D9050008C7080008D9050008EF08000885
:1009D00051060008D905000825090008A086010075
:1009E000703A00082DE9F34702AE00244FF47A75FF
:1009F00006F8014D144FDFF85880454397F9003051
:100A00005A1C5FFA84F901D0A34212D158F824008D
:100A100003680122D3F820A031462B46D047012895
:100A200007D10A4B9DF8070083F8009002B0BDE89B
:100A3000F0870134032CE1D14FF4FA7001F092FAFF
:100A40004FF0FF30F2E700BF002402209829022077
:100A50007C3A00082DE9F0474FF47A75144FDFF81F
:100A6000588006464D43002497F900305A1C5FFA1F
:100A700084F901D0A34210D158F82400036804225D
:100A8000D3F820A031462B46D047042805D1094B86
:100A900083F800900020BDE8F0870134032CE3D1F7
:100AA0004FF4FA7001F05EFA4FF0FF30BDE8F087C6
:100AB00000240220982902207C3A000830B4074B19
:100AC0001A78074B53F822402368DD69054B0A4624
:100AD000AC460146204630BC604700BF9829022042
:100AE0007C3A0008A086010070B501F073FC094C47
:100AF000094E2070002530682378834208D901F020
:100B000063FC336805440133B5F5004F3360F2D31D
:100B100070BD00BF992902207C29022001F022BD6E
:100B200000F1006000F500400068704707B502ABB7
:100B300000F1006043F8041D0422194600F500404E
:100B400001F09EFC03B05DF804FB0000054B1A6841
:100B5000054B1B789B1A834202D9104401F034BC28
:100B6000002070477C2902209929022038B5074DC2
:100B700004462868204401F02FFC28B92868204446
:100B8000BDE8384001F040BC38BD00BF7C290220E0
:100B900010F0030308D1B0F5806F05D800F10050C4
:100BA000A0F571200068704700207047014BC058C5
:100BB000704700BF20F4F01F014B1868704700BF5A
:100BC000002004E0F0B5204B1E68204B1F885D68B4
:100BD00093F90840C6F30B02BA424FEA164622D0F8
:100BE0009F89BA4221D01F8BBA4206D102220C241F
:100BF00004FB02335D6893F90840B6F5805F16D0B8
:100C000041F201039E4208BF5A24421E0A44013D9C
:100C10000B46934215D215F9016F581C4EB103468D
:100C200000F8016CF5E70022E1E70122DFE741244B
:100C3000EBE72C2582421D7001D9981C5C70401A8C
:100C4000F0BD1846FBE700BF002004E004240220AA
:100C5000094B5B88B3F5805F09D041F201029342F2
:100C600007D10122054B03EB8203D878704700229D
:100C7000F8E70020704700BF002004E0743A000845
:100C8000022804D14FF48002034B9A617047012877
:100C9000FCD14FF40002F7E700080240022803D11C
:100CA0004022034B9A6170470128FCD18022F8E76B
:100CB00000080240022805D1064A536983F0400328
:100CC000536170470128FCD1024A536983F08003C5
:100CD000F6E700BF0008024010B50023934203D09E
:100CE000CC5CC4540133F9E710BD000030B5441E9C
:100CF00014F9010F0B4660B193F90050854201F1E0
:100D0000010106D11AB993F90020801A30BD013AC9
:100D1000EEE7002AF7D1104630BD00000246034638
:100D2000981A13F9011B0029FAD1704702440346AF
:100D3000934202D003F8011BFAE77047024B1A787E
:100D4000024B1A70704700BF98290220002402202D
:100D500038B5194C194D204600F04AFC294620466A
:100D600000F072FC2B681648DA6ED2F8043843F0B3
:100D70000203C2F8043801F0F5F81249286800F0BF
:100D80006BFD2B681048DA6E1049D2F8043823F056
:100D90000203C2F80438A0424FF4E1330B6001D0E3
:100DA00000F082FB0A48A04204D00849BDE8384060
:100DB00000F07ABB38BD00BFB4320220703B00089F
:100DC00040420F00C43B00089C29022080290220D9
:100DD000082A022038B50B4B1A780B4B53F82240E7
:100DE0000A4B9C4205460CD0094B0021184618229C
:100DF000FFF79CFF056001462046BDE8384000F043
:100E000053BB38BD982902207C3A0008B432022036
:100E100080290220FEE7000000B59BB0EFF30981B6
:100E200068226846FFF758FFEFF30583034B9A6B80
:100E30009A6A9A6A9A6A9A6A9B6AFEE700ED00E0EB
:100E400000B59BB0EFF3098168226846FFF744FFC5
:100E5000EFF30583034B9A6A9A6A9A6A9A6A9A6AC6
:100E60009B6AFEE700ED00E000B59BB0EFF309815F
:100E700068226846FFF730FFEFF30583034B5A6B98
:100E80009A6A9A6A9A6A9A6A9B6AFEE700ED00E09B
:100E9000026843681143016003B1184770470000BE
:100EA000024A136843F0C0031360704700440040D7
:100EB000024A136843F0C003136070470078004093
:100EC0002DE9F041C66D3768F5693562044628079B
:100ED00019D015F0080F0CBF00218021EA0748BF88
:100EE00041F02001AB0748BF41F04001680748BF0F
:100EF00041F48071202383F31188201DFFF7C8FF80
:100F0000002383F31188E9050AD5202383F3118890
:100F10004FF40071201DFFF7BBFF002383F31188FE
:100F2000AA060CD5202383F31188736A94F8641001
:100F30002046194000F0C6FA002383F311883B06CF
:100F400014D5280612D5202383F3118804F1380024
:100F500000F01EFA002822DA0821201DFFF798FF72
:100F600027F080033360002383F3118879060DD5C1
:100F70006A060BD5202383F31188E26C236D9A4215
:100F800001D1236C6BB9002383F31188EB0610D5D4
:100F9000A26E13696BB15069BDE8F0411847B062A9
:100FA000E1E71021201D27F04007FFF771FF3760B0
:100FB000E9E7BDE8F081000008B50348FFF780FFCE
:100FC000BDE8084001F012BB9C29022008B5034887
:100FD000FFF776FFBDE8084001F008BB082A0220B1
:100FE00037B51F4C1F4D204600F052FA009404F113
:100FF000140000234FF400721B4900F013F94FF462
:101000000072009404F13800184B194900F08CF973
:10101000184BE3652566184C0B21262000F090F84C
:10102000204600F035FA04F11400009400234FF438
:101030000072124900F0F6F804F138000094104BE9
:1010400010494FF4007200F06FF90F4BE3650B216C
:101050005220256603B0BDE8304000F071B800BFF3
:101060009C29022080F93703742A0220A10E00086F
:10107000742E022000440040082A0220742C022012
:10108000B10E00087430022000780040284B00297F
:1010900008BF1946037C8166012B30B50CD1254B66
:1010A000984235D1244B1A6C42F400321A641A6EFD
:1010B00042F400321A661B6E0A68036EC46D03EBBD
:1010C0005203B3FBF2F34A68150442BF23F007054D
:1010D00003F0070343EA4503E3608B6843F04003F2
:1010E0006360CB6843F00103A36042F4967343F05E
:1010F0000103236051054FF0FF33236205D512F041
:10110000102211D0B2F1805F10D080F8643030BD71
:101110000A4B9842D0D1084B1A6C42F080421A64B4
:101120001A6E42F08042C5E77F23EEE73F23ECE7EB
:10113000B43A00089C29022000380240082A022004
:1011400000F1604300F01F02400903F5614309010B
:101150008000C9B200F1604083F8001300F56140DF
:1011600001239340C0F8803103607047F8B51546FD
:1011700082680669AA420B46816938BF8568761A7B
:10118000B542044607D218462A46FFF7A5FDA369D3
:101190002B44A3610DE011D932461846FFF79CFDA0
:1011A000AF1B3A46E1683044FFF796FDE2683A44E7
:1011B000A261A3685B1BA3602846F8BD18462A46B7
:1011C000FFF78AFDE368E4E783682DE9F041044610
:1011D00093421546266938BF85684069361AB5427C
:1011E0000F4606D22A46FFF777FD63692B446361F9
:1011F0000DE012D93246A5EB0608FFF76DFD424619
:10120000B919E068FFF768FDE26842446261A368CB
:101210005B1BA3602846BDE8F0812A46FFF75CFD12
:10122000E368E4E710B50A440024C361029B006050
:1012300040608460C160816141610261036210BDF0
:1012400008B582694369934201D1826882B9826894
:10125000013282605A1C42611970426903699A42E4
:1012600001D3C3684361002100F098FE002008BD4F
:101270004FF0FF3008BD000070B5202304460E4635
:1012800083F31188A568A5B1A368A269013BA36097
:10129000531CA36115782269934224BFE368A361BC
:1012A000E3690BB120469847002383F31188284651
:1012B00070BD3146204600F061FE0028E2DA85F379
:1012C000118870BD2DE9F74F05460F4690469A46A6
:1012D000D0F81C90202686F311884FF0000B14469E
:1012E00064B1224639462846FFF740FF034668B9F5
:1012F0005146284600F042FE0028F1D0002383F337
:101300001188A8EB040003B0BDE8F08FB9F1000F1D
:1013100003D001902846C847019B8BF31188E41A3B
:101320001F4486F31188DBE7C16081614161C361BD
:101330001144009B0060406082600161036270475D
:10134000F8B504460E461746202383F31188A56896
:10135000A5B1A368013BA36063695A1C62611E705A
:10136000236962699A4224BFE3686361E3690BB150
:1013700020469847002080F31188F8BD3946204662
:1013800000F0FCFD0028E2DA85F31188F8BD0000CA
:10139000836942699A4210B501D182687AB982683C
:1013A000013282605A1C82611C7803699A4201D31F
:1013B000C3688361002100F0F1FD204610BD4FF0AD
:1013C000FF3010BD2DE9F74F05460F4690469A466F
:1013D000D0F81C90202686F311884FF0000B14469D
:1013E00064B1224639462846FFF7EEFE034668B947
:1013F0005146284600F0C2FD0028F1D0002383F3B7
:101400001188A8EB040003B0BDE8F08FB9F1000F1C
:1014100003D001902846C847019B8BF31188E41A3A
:101420001F4486F31188DBE70268436811430160BB
:1014300003B11847704700001430FFF743BF0000A6
:101440004FF0FF331430FFF73DBF00003830FFF797
:10145000B9BF00004FF0FF333830FFF7B3BF0000D3
:101460001430FFF709BF00004FF0FF311430FFF7D1
:1014700003BF00003830FFF763BF00004FF0FF32BA
:101480003830FFF75DBF000000207047FFF7A8BDB0
:10149000044B0360002343608360C3600123037433
:1014A000704700BFCC3A000810B52023044683F3F0
:1014B0001188FFF7EBFD02232374002383F31188C7
:1014C00010BD000038B5C36904460D461BB90421A0
:1014D0000844FFF7A9FF294604F11400FFF7B0FE06
:1014E000002806DA201D4FF48061BDE83840FFF780
:1014F0009BBF38BD026843681143016003B11847C0
:101500007047000013B5446BD4F894341A6811780E
:10151000042916D1217C022913D1197912890123BA
:101520008B4013420DD101A904F14C0001F076FE6D
:10153000024630B1D4F89444019B2179206800F030
:10154000DBF902B010BD0000143001F0E5BD000071
:101550004FF0FF33143001F0DFBD00004C3001F0DC
:10156000C9BE00004FF0FF334C3001F0C3BE000095
:10157000143001F0B3BD00004FF0FF31143001F022
:10158000ADBD00004C3001F095BE00004FF0FF32C1
:101590004C3001F08FBE0000D0F8942438B51368A9
:1015A00019780429054601D0012038BD017C0229A3
:1015B000FAD112795C89012090400440F4D105F100
:1015C000140001F045FD02460028EDD0D5F89454F2
:1015D0004FF480732868697900F07CF9204638BDA3
:1015E000406BFFF7D9BF0000002070477047000034
:1015F0007FB5124B0360002343608360C360012505
:1016000002260F4B057404460290019300F18402F8
:10161000294600964FF48073143001F0F5FC094B15
:101620000193029400964FF4807304F523722946C7
:1016300004F14C0001F0CEFD04B070BDF43A000896
:10164000E1150008051500080B68202282F31188B7
:101650000A7903EB820210624A790D3243F82200C4
:101660008A7912B103EB8203186202230374C0F873
:101670009414002383F311887047000038B50446A2
:10168000012502210430FFF735FF04F1140025770E
:101690006FF0010100F08EFC84F8545004F14C000E
:1016A0006FF00101BDE8384000F084BC10B50121A5
:1016B00004460430FFF71EFF0023237784F85430DC
:1016C00010BD000038B504460025143001F0B4FC0C
:1016D00004F14C00257701F095FD201D84F854504D
:1016E0000121FFF707FF2046BDE83840FFF754BF50
:1016F00090F85C3003F06003202B19D190F85D2046
:10170000212A0AD0222A4FF000030ED0202A0FD11E
:10171000084A02650722426504E0064B0365072379
:101720004365002383650120704703654365F9E73E
:101730000020704728240220D0F8943437B51A6866
:101740001178042904461AD1017C022917D119798C
:10175000128901238B40134211D100F14C05284618
:1017600001F026FE58B101A9284601F057FDD4F832
:101770009444019B21790246206800F0BDF803B033
:1017800030BD000000EB8103F7B51C6A05460E462C
:10179000F4B1202383F3118805EB8607201D08216F
:1017A000FFF7A8FEFB685B691B684C3413B1204649
:1017B00001F042FD01A9204601F030FD024648B18A
:1017C000019B3146284600F097F8002383F31188E7
:1017D00003B0F0BDFB685A691268002AF5D01B8A75
:1017E000013B1340F1D105F15C02EAE70D3138B558
:1017F00050F82140DCB1202383F31188D4F89424DD
:101800001368527903EB8203DB689B695D6845B11D
:1018100004216018FFF76EFE294604F1140001F060
:1018200021FC2046FFF7B8FE002383F3118838BD62
:101830007047000000F0D2BF012303700023436013
:1018400000F1240200F1380142F8043B8A4213619E
:10185000FAD103814381704738B50446202383F3CE
:10186000118800254160C560056145618561C561DC
:10187000056200F0C3FF0223237085F3118838BD91
:1018800070B500EB810305465069DA600E461446D8
:1018900018B110220021FFF749FAA06918B11022EF
:1018A0000021FFF743FA31462846BDE8704001F0B9
:1018B0006BB80000028902F001020281428902F045
:1018C000010242810022026142618261C2610262C0
:1018D00001F0EEB8F0B400EB81044789E46801251B
:1018E000A4698D403D43458123600023A26063606D
:1018F000F0BC01F009B90000F0B400EB81040789E5
:10190000E468012564698D403D430581236000231F
:10191000A2606360F0BC01F083B9000070B50223DF
:10192000002504460370A0F8645080F8665080F8E3
:10193000675005814581C560056145618561C56167
:10194000056280F84C5000F0BBFF63681B6823B150
:1019500029462046BDE87040184770BD43680278AC
:101960001B6880F86820052202700BB1042118471B
:1019700070470000436890F868201B6802700BB144
:10198000052118477047000090F84C3070B50446A8
:1019900013B1002380F84C3004F15C02204601F0C2
:1019A000A9F863689B6863BB94F85C5015F0600607
:1019B00015D194F85D3005F07F0545EA032540F226
:1019C00002339D4200F00E815BD8022D00F0DC80D6
:1019D0003FD8002D00F08780012D00F0CF8000213E
:1019E000204601F0F3FA0021204601F0E5FA636891
:1019F0001B6813B1062120469847062384F84C3013
:101A000070BD204698470028CED094F8632094F803
:101A1000623043EA0223626D934238BF636594F9F2
:101A20005C30656D002B4FF0200380F2FD80002DAF
:101A300000F0EC80092284F84C2083F31188002107
:101A4000636D226D2046FFF757FF002383F3118853
:101A500070BDB5F5817F00F0B180B5F5407F49D00C
:101A6000B5F5807FBBD194F85E30012BB7D1B4F8C7
:101A7000643023F00203A4F8643026656665A66529
:101A8000C3E740F201639D421ED8B5F5C06F3BD25B
:101A9000B5F5A06FA3D1B4F85C30B3F5A06F0ED14B
:101AA00094F85E3084F86630204600F061FF636889
:101AB0001B6813B10121204698470323237000239C
:101AC00023656365A365A0E7B5F5106F32D040F6D6
:101AD00002439D4252D0B5F5006F80D104F16703F7
:101AE0002365012324E004F1640323650223636575
:101AF000A5658AE794F85E30012B7FF470AFB4F8E7
:101B0000643043F00203B6E794F86120616894F80A
:101B100060304D6894F85F1043EA0223204694F841
:101B20005E20A84700283FF45AAF43682365036846
:101B30006365A4E72378042B10D1202383F3118855
:101B40002046FFF7B7FE86F31188636884F8676064
:101B50001B68032121700BB12046984794F85E3032
:101B6000002BACD084F867300423237063681B68B3
:101B7000002BA4D0022120469847A0E7374B2365CD
:101B80000223636500239DE794F8601011F0800F35
:101B9000204601F00F010ED000F09EFF012806D074
:101BA00002287FF41CAF2E4B2365606567E72D4B41
:101BB0002365656563E700F081FFEFE794F85E3029
:101BC000002B7FF40CAF94F8603013F00F013FF45A
:101BD00076AF1A06204602D501F00CFA6FE701F045
:101BE000FFF96CE794F85E30002B7FF4F8AE94F8C0
:101BF000603013F00F013FF462AF1B06204602D5A0
:101C000001F0E4F95BE701F0D7F958E7142284F812
:101C10004C2083F311882B462A4629462046FFF79D
:101C200059FE85F3118870BD5DB1152284F84C20F2
:101C300083F311880021636D226D2046FFF74AFE71
:101C400003E70B2284F84C2083F311882B462A46A5
:101C500029462046FFF750FEE3E700BF243B00087B
:101C60001C3B0008203B000838B590F84C30044677
:101C7000152B29D8DFE803F03E28282828283E28FD
:101C8000280B293928282828282828283E3E90F87B
:101C9000631090F86220436D42EA01229A4214D9FF
:101CA000C268128AB3FBF2F502FB15356DB9202329
:101CB00083F311882B462A462946FFF71DFE85F33C
:101CC00011880A2384F84C3038BD142384F84C3032
:101CD000202383F3118800231A4619462046FFF774
:101CE000F9FD002383F3118838BD836D03B1984754
:101CF0000023E7E7002101F069F90021204601F007
:101D00005BF963681B6813B10621204698470623D8
:101D1000D8E7000090F84C20152A38B5044622D8A0
:101D20000123934040F6416213421DD113F4801504
:101D30000FD19B0217D50B2380F84C30202383F35F
:101D400011882B462A462946FFF7D6FD85F31188D0
:101D500038BDC3689B695B682BB9836D03B1984735
:101D6000002384F84C3038BD002101F02FF9002108
:101D7000204601F021F963681B6813B10621204653
:101D800098470623EDE70000024B00221B605B60D2
:101D90009A60704774320220002303748268054BF6
:101DA0001B6899689142FBD25A68036042601060D8
:101DB000586070477432022008B5202383F31188DD
:101DC000037C032B05D0042B0DD02BB983F3118892
:101DD00008BD436900221A604FF0FF334361FFF7EB
:101DE000DBFF0023F2E790E80C001A600268536002
:101DF000F2E70000002303748268054B1B689968B2
:101E00009142FBD85A680360426010605860704786
:101E100074320220054B19690874186802681A6048
:101E20005360186101230374FEF77EBA74320220F6
:101E300030B54B1C87B005460A4C10D023690A4ABE
:101E400001A800F0D3F82846FFF7E4FF049B13B184
:101E500001A800F007F92369586907B030BDFFF702
:101E6000D9FFF8E774320220B91D000838B50C4DCF
:101E700041612B6981689A689142044603D8BDE8A4
:101E80003840FFF789BF1846FFF786FF01232C6112
:101E9000014623742046BDE83840FEF745BA00BF2E
:101EA00074320220044B1A681B6990689B68984240
:101EB00094BF0020012070477432022010B5084CF6
:101EC000236820691A6822605460012223611A7411
:101ED000FFF790FF01462069BDE81040FEF724BAE5
:101EE000743202208260022202740022427470471F
:101EF0008368A3F17C0243F80C2C026943F83C2C64
:101F0000426943F8382C074A43F81C2CC26843F84E
:101F1000102C022203F8082C002203F8072CA3F14E
:101F2000180070474103000810B5202383F311887F
:101F3000FFF7DEFF00210446FFF798FF002383F33D
:101F40001188204610BD0000024B1B6958610F200C
:101F5000FFF760BF74320220202383F31188FFF75C
:101F6000F3BF000008B50146202383F31188082041
:101F7000FFF75EFF002383F3118808BD49B1064BCC
:101F800042681B6918605A60136043600420FFF7C1
:101F90004FBF4FF0FF307047743202200368984201
:101FA00006D01A680260506059611846FFF7F4BE07
:101FB0007047000038B504460D462068844200D1C1
:101FC00038BD036823605C604561FFF7E5FEF4E718
:101FD000054B03F114025A619A614FF0FF32DA6146
:101FE00000221A62704700BF74320220F8B5036104
:101FF0004FF08043C2605C6A194B1A46022952F8BE
:10200000145F38BF0221954206461F460AD1586127
:1020100098611C620560456081600819BDE8F84060
:1020200001F0E8B9186AAB68241A0C1902D3E41A53
:102030002D6804E09C4202D2204401F0E9F9AB682B
:102040009C42F4D86B68736035601E606E60B4604B
:10205000A9684FF0FF33091BA960FB61F8BD00BF01
:102060007432022010B41B4C234653F8141F8142D3
:1020700010D0416802680A60026851609A424FF0CD
:102080000001C16003D0936881680B4493605DF8E0
:10209000044B70470A68626100209A425360C8602E
:1020A00003D15DF8044B01F0ADB99368886803442F
:1020B00093604FF08042206A526A121A9342E6D926
:1020C000991A012998BF931C18445DF8044B01F03C
:1020D0009FB900BF7432022000207047FEE7000065
:1020E000704700004FF0FF3070470000022906D013
:1020F000032906D00129064818BF0020704705486B
:102100007047032A9ABF044800EBC20000207047C2
:10211000203C0008D43B00083024022070B504465F
:1021200008460D46FEF7FAFDC6B220460134037894
:102130000BB9184670BD32462946FEF7D7FD002878
:10214000F3D1012070BD00002DE9F04F80469BB017
:1021500008460C461646FEF7E1FD3C49C5B220464E
:10216000FFF7DCFF08B10735EDB239492046FFF72C
:10217000D5FF08B11035EDB2632D01AF0CD8DFF8F3
:10218000DC90DFF8DCB03D4694F800A0BAF1000F17
:102190001CD185F800A003E02146384601F05EFC22
:1021A0003846FEF7BBFDC0B2431C5B0088E8480020
:1021B000337003237370002302361946DAB290425B
:1021C00006F102063BD81BB0BDE8F08FBAF1250F2F
:1021D00030D107221D492046FEF788FD70B91D4BFE
:1021E0002A4603F10C0153F8040B42F8040B8B420E
:1021F000F9D11B88138007340E35C5E7082214492E
:102200002046FEF773FDA8B91349AB1C11F8012F46
:10221000100902F00F0210F8090012F8092003F863
:10222000020C594503F8012C03F10203EED11835D5
:102230000834A9E785F800A001340135A4E7FA5C69
:1022400006F8022C06F8011C0133B7E7783B0008BA
:10225000803B0008893B00081FF4F01F983B0008F2
:102260002BF4F01F08B5202383F311880348FFF7F0
:1022700063FA002383F3118808BD00BFB432022043
:1022800010B50446052916D8DFE801F01615031627
:10229000161D202383F311880E4A0121FFF7F0FA5F
:1022A00020460D4A0221FFF7EBFA0C48FFF70AFA25
:1022B000002383F3118810BD202383F3118807487E
:1022C000FFF7DCF9F4E7202383F311880348FFF7D5
:1022D000EDF9EDE7283B00084C3B0008B432022042
:1022E00038B50C4D0C4C0D492A4604F10800FFF797
:1022F0002BFF05F1CA0204F110000949FFF724FF82
:1023000005F5CA7204F118000649BDE83840FFF728
:102310001BBF00BF7C37022030240220AC3B0008EA
:10232000B63B0008803B0008BFF34F8F024AD368DA
:10233000DB03FCD4704700BF003C024008B5074BEC
:102340001B7853B9FFF7F0FF054B1A69002ABFBF8E
:10235000044A5A6002F188325A6008BDDA39022014
:10236000003C02402301674508B5054B1B7833B993
:10237000FFF7DAFF034A136943F00043136108BD16
:10238000DA390220003C02400B2870B513D80B4A02
:102390000B4C137863B90B4E4FF0006144F82310D7
:1023A00056F8235001330C2B2944F7D10123137025
:1023B00054F8200070BD002070BD00BF0C3A022010
:1023C000DC390220403C0008014B53F820007047E4
:1023D000403C00080C2070470B2810B5044601D97A
:1023E000002010BDFFF7D0FF064B53F824301844EF
:1023F000C21A0BB9012010BD12680132F0D1043BA2
:10240000F6E700BF403C00080B2810B504462FD863
:10241000FFF78AFFFFF792FF1649F323CB60FFF720
:1024200083FFC300DBB243F4007343F002030B618C
:102430000B6943F480330B61FFF776FFFFF7A4FFCE
:102440000D4B53F824300344BFF34F8F0B4A98428F
:102450000AD3BFF34F8FBFF36F8FFFF785FF20467F
:10246000BDE81040FFF7B8BFC2F85C022030EEE7CD
:10247000002010BD003C0240403C000800ED00E0A0
:102480002DE9F047D40715464DD41318B3F1026F68
:1024900049D2324B1B68DA0745D5314CFFF74EFF66
:1024A000F323E360FFF740FF2F46401A40F2012973
:1024B000032F884601EB000618D8294C40F2011979
:1024C0007B1A4344012B01EB000623692FD823F02C
:1024D00001032361FFF748FF2846BDE8F08736680F
:1024E00051F8043CB34218D1043FE1E7B307E4D10B
:1024F000236923F440732361236943EA09032361B9
:102500000431D8F800303360BFF34F8FFFF70CFF72
:10251000E368002BE3D0F323E360236923F0010396
:102520002361FFF721FF4FF0FF30BDE8F08723F470
:1025300040732361236943EA090323618A4631F822
:10254000023B3380BFF34F8FFFF7EEFE3688BAF8B9
:102550000030B6B2B342B3D0DFE700BF003802406C
:10256000003C0240084908B50B7828B153B9FFF781
:10257000E5FE01230B7008BD23B1BDE808400870DB
:10258000FFF7F2BE08BD00BFDA390220014B186D1B
:10259000704700BF00280040094B1A6F120407D48F
:1025A0001A6F42F400721A671A6F42F400421A67F7
:1025B000044A136843F480731360034B1865704733
:1025C000003802400070004000280040064A53686E
:1025D00023F001035360EFF30983683383F3098821
:1025E000002383F31188704730EF00E010B52023FB
:1025F00083F31188104B5B6813F4006318D0F1EE7D
:10260000103AEFF309844FF0807344F84C3C0B4BC5
:10261000DB6844F8083CA4F1680383F30988FFF7FA
:1026200041FC18B1064B44F8503C10BD054BFAE78D
:1026300083F3118810BD00BF00ED00E030EF00E033
:102640005103000854030008F0B5BFF34F8FBFF3E8
:102650006F8F1D4B0021C3F85012BFF34F8FBFF394
:102660006F8F5A6942F400325A61BFF34F8FBFF344
:102670006F8FC3F88410BFF34F8FD3F88020C2F35D
:10268000C904C2F34E325201A50743F6E07602EACE
:10269000060E284621464EEA00070139C3F860724B
:1026A0004F1C00F14040F6D1203A12F1200FEED13C
:1026B000BFF34F8F5A6942F480325A61BFF34F8F94
:1026C000BFF36F8FF0BD00BF00ED00E0FEE700003C
:1026D000084A094B09498B4204D3094A0021934215
:1026E00005D3704752F8040F43F8040BF3E743F89F
:1026F000041BF4E74C3E0008183D0220183D022060
:10270000183D0220036F30B500229D68C46E11464B
:102710004FF0FF3004EB421301329542C3F8001929
:10272000C3F81019C3F80809C3F8001BC3F8101B3D
:10273000C3F8080BEED24FF00113C4F81C3830BDBB
:10274000890141F02001016103699B06FCD412203C
:1027500000F0ECBE204B03EB80022DE9F047D2F8ED
:102760000CE0DD6EDEF81420461CD2F800C005EB4C
:10277000063605EB4018516861450BD3D5F834286F
:10278000012303FA00F022EA0000C5F834081846D5
:10279000BDE8F087BEF81040ACEB0103A34228BFB0
:1027A0002346D8F81849A4B2B3EB840F10D8946824
:1027B0001F46A4F1040959F804AFC6F800A0042F7D
:1027C00001D9043FF7E71C440B4494605360D2E7FF
:1027D0000020BDE8F08700BF103A022010B5054C7C
:1027E0002046FFF729F84FF0A043E366024B23672A
:1027F00010BD00BF103A0220943C00080378012B62
:1028000070B505464DD1284BC46E98421BD1274B5D
:102810005A6B42F080025A635A6D42F080025A6548
:102820005A6D5A6942F080025A615A6922F0800258
:102830005A610E2143205B69FEF782FC1C4BE3606A
:102840001C4BC4F800380023C4F8003EC0232360AA
:102850004FF40413A363EE6E202000F067FE012303
:1028600033613369DB07FCD4122000F05FFE33696B
:10287000002BFCDA0026A6602846FFF743FF6B68B2
:10288000C4F81068DB68C4F81468C4F81C684BB955
:10289000094BA3614FF0FF336361A36843F0010369
:1028A000A36070BD054BF4E7103A022000380240E7
:1028B0004014004003002002003C30C0083C30C0FF
:1028C000F8B5C46E054600212046FFF739FF296F91
:1028D00000234FF001128F68C4F834384FF00066BF
:1028E000C4F81C284FF0FF3004EB431201339F4221
:1028F000C2F80069C2F8006BC2F80809C2F8080BF8
:10290000F2D20B68EA6E6B6763621023136116697B
:1029100016F01006FBD1122000F008FED4F80038A3
:1029200023F4FE63C4F80038A36943F4402343F062
:102930001003A3610923C4F81038C4F814380A4BF3
:10294000EB604FF0C043C4F8103B084BC4F8003BA9
:10295000C4F81069C4F800396B6F03F1100243F436
:1029600080136A67A362F8BD703C000840800010C5
:10297000C26E90F86610D2F8003823F4FE6343EA82
:102980000113C2F8003870472DE9F0410EB200EB98
:1029900086080D46D8F80C100F6807F00303022BC9
:1029A00050D0032B50D03D4A3D4F012B18BF174646
:1029B000C46E4FEA451E04EB0E030022C3F8102B31
:1029C0008A6905F1100C002A40D04A8A05F15803A3
:1029D0005B013A43E2500123D4F81C2803FA0CF3BC
:1029E0001343A6444A69C4F81C380023CEF81039B2
:1029F00005F13F03002A39D00A8A898B9208012900
:102A000088BF4A43416F04EB8303561841EA0242F0
:102A1000466729465A602046FFF792FED8F80C30E8
:102A20001B8A43EA85531F4305F148035B01E750C6
:102A30000123D4F81C2803FA05F51543C4F81C58E3
:102A4000BDE8F081174FB3E7174FB1E704EB46132A
:102A5000D3F8002B22F40042C3F8002BD4F81C2832
:102A6000012303FA0CF322EA0303BAE704EB83031E
:102A70000E4A5A6004EB461629462046FFF760FED0
:102A8000D6F8003923F40043C6F80039D4F81C38CE
:102A9000012202FA05F523EA0505CFE700800010C0
:102AA000008004100080081000800C100004000258
:102AB000026F12684267FFF725BE00005831C36EEF
:102AC00049015B5813F4004004D013F4001F14BFF5
:102AD00001200220704700004831C36E49015B5855
:102AE00013F4004004D013F4001F14BF012002208F
:102AF0007047000000EB8101CB68196A0B68136016
:102B00004B6853607047000000EB810330B5DD680F
:102B1000AA691368D36019B9402B84BF402313609E
:102B20006B8A1468C26E1C44013CB4FBF3F463432B
:102B3000033323F0030302EB411043EAC44343F0A1
:102B4000C043C0F8103B2B6803F00303012B09B20C
:102B50000ED1D2F8083802EB411013F4807FD0F880
:102B6000003B14BF43F0805343F00053C0F8003BD8
:102B700002EB4112D2F8003B43F00443C2F8003BA1
:102B800030BD00002DE9F041244DEE6E06EB401300
:102B90000446D3F8087BC3F8087B38070AD5D6F873
:102BA0001438190706D505EB84032146DB6828464F
:102BB0005B689847FA072FD5D6F81438DB072BD572
:102BC00005EB8403D968CCB98B69488A5E68B6FB8B
:102BD000F0F200FB12628AB91868DA6890420DD2EE
:102BE000121A83E81400202383F311880B4821462E
:102BF000FFF78AFF84F31188BDE8F081012303FA0F
:102C000004F26B8923EA02036B81CB6823B121466E
:102C10000248BDE8F0411847BDE8F081103A0220B3
:102C200000EB810370B5DD68C36E6C692668E660F1
:102C30004A0156BB1A444FF40020C2F810092A6812
:102C400002F00302012A0AB20ED1D3F8080803EBFE
:102C5000421410F4807FD4F8000914BF40F0805073
:102C600040F00050C4F8000903EB4212D2F800090A
:102C700040F00440C2F80009D3F83408012202FAF7
:102C800001F10143C3F8341870BD19B9402E84BF57
:102C90004020206020682E8A841940F00050013CBA
:102CA0001A44B4FBF6F440EAC440C6E7F8B504465B
:102CB0001E48C56E05EB4413D3F80869C3F80869CC
:102CC000F10717D5D5F81038DA0713D500EB8403D0
:102CD000D9684B691F68DA68974218D2D21B00275F
:102CE0001A605F60202383F311882146FFF798FF65
:102CF00087F31188330617D5D5F834280123A3406C
:102D0000134211D02046BDE8F840FFF723BD012350
:102D100003FA04F2038923EA020303818B68002B80
:102D2000E8D021469847E5E7F8BD00BF103A0220F9
:102D3000A0482DE9F84FC56E6E69AB691E4016F4C8
:102D4000805F6E61044605D0FEF7E8FDBDE8F84FF0
:102D5000FFF74CBC002E12DAD5F8003E95489B07D1
:102D60001EBFD5F8003E23F00303C5F8003ED5F89A
:102D7000043823F00103C5F80438FEF7FBFD3705DE
:102D800002D58C48FEF7EAFDB0040CD5D5F808381A
:102D900013F0060FEB6823F470530CBF43F4105389
:102DA00043F4A053EB60310704D56368DB680BB1D3
:102DB00080489847F2026FD4B3020CD5D4F86C80E7
:102DC000DFF8F0A100274FF00109236F9B68F9B2EB
:102DD0008B4280F09C80F70619D5E16E0A6AC2F337
:102DE0000A1702F00F0302F4F012B2F5802F00F080
:102DF000B680B2F5402F0AD104EB830301F5805170
:102E0000DB68186A00231A469F4240F09C80330317
:102E1000D5F818481DD5E70302D50020FFF7B2FE0C
:102E2000A50302D50120FFF7ADFE600302D5022005
:102E3000FFF7A8FE210302D50320FFF7A3FEE2025D
:102E400002D50420FFF79EFEA30202D50520FFF75E
:102E500099FE77037FF57AAFE60702D50020FFF7EA
:102E600025FFA50702D50120FFF720FF600702D547
:102E70000220FFF71BFF210702D50320FFF716FFF3
:102E8000E20602D50420FFF711FFA3067FF55EAF2F
:102E90000520FFF70BFF59E7D4F86C80DFF814A189
:102EA00000274FF00109236F9B685FFA87FB5B45A2
:102EB00082D308EB4B13D3F8002902F44022B2F579
:102EC000802F22D1D3F80029002A1EDAD3F8002956
:102ED00042F09042C3F80029D3F80029002AFBDB16
:102EE0005946E06EFFF72CFC228909FA0BF322EA1F
:102EF0000303238104EB8B03DB689B6813B1594602
:102F0000504698475846FFF725FC0137CBE708EBBA
:102F10004112D2F8003B03F44023B3F5802F10D1C7
:102F2000D2F8003B002B0CDA628909FA01F322EA9D
:102F30000303638104EB8103DB68DB680BB150465C
:102F40009847013741E79C0708BF0A68072B98BFDD
:102F5000027003F101039CBF120A013054E70233EF
:102F600004EB830201F58051526890690268D0F841
:102F700008C04068A2EB000E0022104697420AD11A
:102F800004EB830463689B699A683A449A605A68C0
:102F900017445F603BE712F0030F08BF08689645CF
:102FA00088BF8CF8000002F1010284BF000A0CF116
:102FB000010CE3E7103A0220C36E03EB4111D1F894
:102FC000003B43F40013C1F8003B7047C36E03EBB2
:102FD0004111D1F8003943F40013C1F800397047AA
:102FE000C36E03EB4111D1F8003B23F40013C1F889
:102FF000003B7047C36E03EB4111D1F8003923F455
:103000000013C1F80039704730B5039C01720433D6
:1030100004FB0325C361049B03630021059B00603F
:103020004060C16042610261856104624262816206
:10303000C162436330BD00000022416A4161016109
:10304000C2608262C2626FF00101FEF7B3BF00008E
:1030500003694269934203D1C2680AB100207047F4
:10306000181D704703691960C2680132C260C269E5
:10307000134482690361934224BF436A03610021C0
:10308000FEF78CBF38B504460D46E3683BB1626974
:10309000131D1268A3621344E362002038BD237A33
:1030A00033B929462046FEF769FF0028EDDA38BD1E
:1030B0006FF00100FBE70000C368C269013BC36019
:1030C0004369134482694361934224BF436A436165
:1030D00000238362036B03B11847704770B5202348
:1030E000044683F31188866A3EB9FFF7CBFF054695
:1030F00018B186F31188284670BDA36AE26A13F8F6
:10310000015BA362934202D32046FFF7D5FF002361
:1031100083F31188EFE700002DE9F74F1F460446BF
:103120000E469146202383F311884FF080480025F6
:10313000D8F82430FB18009307F1FF3AAB46A36A96
:10314000ABB91AF1030F06D939462046FFF79AFFAB
:1031500068B1002305E0D8F82410009A511A8F4274
:10316000F3D283F31188284603B0BDE8F08FA16A3B
:10317000E36AA9EB05025B1A934228BF1346402B72
:103180001CD9334601F1400251F8040B43F8040BFB
:103190009142F9D1A36A40334036A3624035A26A16
:1031A000E36A9A4202D32046FFF786FF8BF3118829
:1031B0004D45D8D2202383F31188C0E71A46304604
:1031C0000193FDF789FD019BA26A1A441E44A26285
:1031D0001D44E4E710B5029C0172043303FB042193
:1031E000C36100238362C362039B0363049B00608B
:1031F0004060C46042610261816104624262436373
:1032000010BD0000026AC260426A4261026100228F
:103210008262C2626FF00101FEF7CCBE43690269AF
:103220009A4203D1C2680AB100207047184650F88C
:10323000043B0B6070470000C368C2690133C36080
:103240004369134482694361934224BF436A4361E3
:103250000021FEF7A3BE000038B504460D46E36822
:103260003BB123691A1DA262E2691344E3620020A4
:1032700038BD237A33B929462046FEF77FFE002861
:10328000EDDA38BD6FF00100FBE70000036919605B
:10329000C268013AC260C269134482690361934201
:1032A00024BF436A036100238362036B03B11847A1
:1032B0007047000070B5202304460E4683F3118842
:1032C000856A35B91146FFF7C7FF10B185F311883C
:1032D00070BDA36A1E70A36AE26A01339342A362BF
:1032E00004D3E16920460439FFF7D0FF002080F3C2
:1032F000118870BD2DE9F74F1F4604460D469146D3
:10330000202383F311884FF080480026D8F824301A
:10331000FB18009307F1FF3AB346A36AABB91AF161
:10332000030F06D939462046FFF796FF68B1002300
:1033300005E0D8F82410009A511A8F42F3D283F393
:103340001188304603B0BDE8F08FA06AE36AA9EBAC
:1033500006021B1A934228BF1346402B1CD905F1C5
:10336000400355F8042B40F8042B9D42F9D1A36A81
:103370004033A3624036A26AE36A9A4204D3E16909
:1033800020460439FFF782FF8BF311884E45D8D2CF
:10339000202383F31188C0E71A4629460193FDF7DD
:1033A0009BFC019BA26A1A441D44A2621E44E2E7F0
:1033B000026943699A4203D1C3681BB91846704732
:1033C0000023FBE7836A002BF8D0043B9B1AF5D05F
:1033D0001360C368013BC360C3691A448369026117
:1033E0009A4224BF436A0361002383620123E5E715
:1033F00000F040B94FF08043002258631A61022266
:10340000DA6070474FF080430022DA6070470000B6
:103410004FF0804358637047FEE7000010B5194C29
:10342000FEF7B2FCFEF7D4FD802217492046FEF7D6
:1034300059FD012344F8180C0374144B144AD9683D
:1034400021F4E0610904090C0A431249DA60CA68F0
:1034500042F08072CA60104A1049C2F8B01F116869
:1034600041F0010111601022DA77202283F8222036
:10347000002383F3118862B60948BDE81040FEF7C7
:1034800053BD00BF9C320220A03C000800ED00E0CC
:103490000003FA05F0ED00E0001000E055CEACC5E9
:1034A000A83C00082DE9F84F1F4C4FF00008656953
:1034B00004F11407C1464FF08043266A5B6AAA688C
:1034C0009E1B96421DD34FF0200AAA68236AD5F8A6
:1034D0000CB0134423622B68BB425F60A6EB02066C
:1034E0006361C5F80C8001D1FFF78CFF89F3118867
:1034F0002869D8478AF311886569AB689E42E4D28F
:10350000D9E76269BA420CD0916823628E1B96603B
:10351000A86802282CBF1818981CBDE8F84FFFF7C0
:1035200077BFBDE8F88F00BF74320220034B5968A3
:103530005A68521A9042FBD8704700BF001000E052
:103540004B6843608B688360CB68C3600B694361E1
:103550004B6903628B6943620B680360704700002C
:1035600008B5274B27481A6940F2FF710A431A61D0
:103570001A6922F4FF6222F007021A611A691A6BB3
:103580000A431A631A6D0A431A651F4A1B6D1146D6
:10359000FFF7D6FF1D4802F11C01FFF7D1FF1C48C1
:1035A00002F13801FFF7CCFF1A4802F15401FFF78E
:1035B000C7FF194802F17001FFF7C2FF174802F177
:1035C0008C01FFF7BDFF164802F1A801FFF7B8FF15
:1035D000144802F1C401FFF7B3FF134802F1E00100
:1035E000FFF7AEFF114802F1FC01FFF7A9FF1048F9
:1035F00002F58C71FFF7A4FFBDE8084000F09CB80D
:103600000038024000000240C83C000800040240AC
:1036100000080240000C024000100240001402406A
:1036200000180240001C024000200240002402401A
:103630000028024008B500F0F3F9FFF7EFFEBDE8FF
:103640000840FEF74DBE0000704700004FF0804379
:1036500010B51A69920708D500241C61202383F352
:103660001188FFF71FFF84F31188BDE81040FEF7B3
:10367000BDBF0000104B1A6C42F001021A641A6EB2
:1036800042F001021A660D4A1B6E936843F0010373
:1036900093604FF080436B229A624FF0FF32DA6200
:1036A00000229A615A63DA605A6001225A61082145
:1036B0001A601C20FDF744BD00380240002004E0E1
:1036C0001B4B1A696FEA42526FEA52521A611A6929
:1036D000C2F30A021A614FF0FF301A695A69586141
:1036E00000215A6959615A691A6A62F080521A6255
:1036F0001A6A02F080521A621A6A5A6A58625A6A40
:1037000059625A6A0B4A106840F480701060186F52
:1037100000F44070B0F5007F1EBF4FF48030186792
:103720001967536823F40073536000F059B900BF60
:103730000038024000700040354B364A1A64364A61
:103740004FF4404111601A6842F001021A601A6891
:103750009207FCD59A6822F003029A602C4B194616
:103760009A6812F00C02FBD1186800F0F90018609A
:103770009A601A6842F480321A600B689B03FCD589
:103780004B6F43F001034B67214B5A6F9007FCD5F9
:10379000224A5A601A6842F080721A601E4B1A461A
:1037A00059684904FCD5196841F48031196053689F
:1037B000D803FCD5136843F400331360164A5368EA
:1037C0009903FCD5124B1A689201FCD5144A9A60F1
:1037D00040F20112C3F88C200022C3F89020114A55
:1037E00040F2073111609A6842F002029A60084B79
:1037F0009A6802F00C02082AFAD15A6C42F480420C
:103800005A645A6E42F480425A665B6E704700BF3B
:1038100000380240000400100070004008364009E3
:1038200000948838003C0240084A08B55369116882
:103830000B4003F00103536123B1054A13680BB138
:1038400050689847BDE80840FEF7D0BE003C0140F4
:10385000983C0220084A08B5536911680B4003F0F0
:103860000203536123B1054A93680BB1D0689847AE
:10387000BDE80840FEF7BABE003C0140983C02207B
:10388000084A08B5536911680B4003F004035361FB
:1038900023B1054A13690BB150699847BDE8084048
:1038A000FEF7A4BE003C0140983C0220084A08B53F
:1038B000536911680B4003F00803536123B1054AB3
:1038C00093690BB1D0699847BDE80840FEF78EBEFA
:1038D000003C0140983C0220084A08B55369116831
:1038E0000B4003F01003536123B1054A136A0BB177
:1038F000506A9847BDE80840FEF778BE003C01409A
:10390000983C0220174B10B55C691A68144004F407
:1039100078725A61A30604D5134A936A0BB1D06A30
:103920009847600604D5104A136B0BB1506B98474B
:10393000210604D50C4A936B0BB1D06B9847E20576
:1039400004D5094A136C0BB1506C9847A30504D5F4
:10395000054A936C0BB1D06C9847BDE81040FEF758
:1039600045BE00BF003C0140983C02201A4B10B5F8
:103970005C691A68144004F47C425A61620504D5FB
:10398000164A136D0BB1506D9847230504D5134AA1
:10399000936D0BB1D06D9847E00404D50F4A136EB8
:1039A0000BB1506E9847A10404D50C4A936E0BB12D
:1039B000D06E9847620404D5084A136F0BB1506F5C
:1039C0009847230404D5054A936F0BB1D06F9847ED
:1039D000BDE81040FEF70ABE003C0140983C0220C2
:1039E000062108B50846FDF7ABFB06210720FDF7C9
:1039F000A7FB06210820FDF7A3FB06210920FDF700
:103A00009FFB06210A20FDF79BFB06211720FDF7EF
:103A100097FB06212820BDE80840FDF791BB000078
:103A200008B5FFF74DFE00F00DF8FDF72FFDFDF78F
:103A300001FFFDF7DBFDFFF707FEBDE80840FFF7DC
:103A4000D7BC0000002304491A465A50C81808334E
:103A5000802B4260F9D17047983C0220034611F850
:103A6000012B03F8012B002AF9D170471210121311
:103A7000121100000010410001105A00B43202205F
:103A80009C290220082A022053544D3332463F3FDE
:103A90003F3F3F3F0053544D333246375B347C3514
:103AA0005D780053544D333246375B367C375D7852
:103AB0000000000000960000000000000000000070
:103AC00000000000000000000000000000000000F6
:103AD00055140008411400087D14000869140008FA
:103AE00075140008611400084D140008391400080A
:103AF0008914000800000000651500085115000831
:103B00008D15000879150008851500087115000845
:103B10005D15000849150008E915000800000000BF
:103B20000100000000000000020000000000000092
:103B300085170008ED170008400040004C370220B0
:103B40005C370220020000000000000003000000BB
:103B50000000000031180008000000001000000004
:103B60006C3702200000000001000000000000008F
:103B7000103A02200101020025424F415244250023
:103B80002553455249414C25005442532D436F6CF7
:103B9000696272692D463700303132333435363739
:103BA0003839414243444546000000004172647583
:103BB00050696C6F740025424F415244252D424C90
:103BC0000000000081220008ED200008F116000826
:103BD0006522000843000000DC3B000809024300A6
:103BE000020100C0320904000001020201000524A4
:103BF000001001052401000104240202052406002E
:103C000001070582030800FF09040100020A000001
:103C10000007050102400000070581024000000086
:103C200012000000283C00081201100102000040B0
:103C30008304405700020102030100000403090449
:103C40000080000000800000008000000080000074
:103C50000000020000000400000004000000040056
:103C60000000040000000400000004000000040044
:103C70000000000089190008691C0008151D0008D3
:103C800040004000883A0220883A022001000000EB
:103C9000983A02208000000040010000050000006A
:103CA0006D61696E00000000C03C0008A03A02206F
:103CB000983C0220010000001934000800000000B8
:103CC00069646C65000000000000802A00000000AC
:103CD000AAAAAAAA00000000FFFF0000000000003E
:103CE00000A00A000000000000000000AAAAAAAA82
:103CF00000000000FFFF00000000000000000000C6
:103D00000050000000000000AAAAAAAA00000000BB
:103D1000FFFF0000000000000000000080290000FC
:103D200000000000AAAAAAAA40150000FFFF000098
:103D3000007070070000000040000200000000005A
:103D4000AAAAAAAA00000100F7FF000000000000D4
:103D5000080000000020000000000000AAAAAAAA93
:103D600000100000FFFF000000000008000000003D
:103D70000040000000000000AAAAAAAA000000005B
:103D8000FFFF000000000000000000000000000035
:103D900000000000AAAAAAAA00000000FFFF00007D
:103DA0000000000000000000000000000000000013
:103DB000AAAAAAAA00000000FFFF0000000000005D
:103DC00000000000000000000000000000000000F3
:103DD00000000000000000000000000000000000E3
:103DE00000000000000000000000000000000000D3
:103DF00000000000000000000000000000000000C3
:103E0000FF00000000000000883A00083F000000AA
:103E100049040000953A00083F00000051040000EA
:103E2000A33A00083F0000000096000000000800D0
:103E3000040000003C3C00080000000000000000FE
:103E40000000000000000000000000000000000072
:00000001FF
